S02B00002F686F6D652F766F6F72627572672F446576656C6F706D656E742F4F70656E424C542F5461726765E0
S3150800200000300020F52E0008452F0008452F00084F
S31508002010452F0008452F0008452F0008000000003E
S31508002020000000000000000000000000452F000826
S31508002030452F000800000000452F0008A52F0008BE
S31508002040452F0008452F0008452F0008452F000892
S31508002050452F0008452F0008452F0008452F000882
S31508002060452F0008452F0008452F0008452F000872
S31508002070452F0008452F0008452F0008452F000862
S31508002080452F0008452F0008452F0008452F000852
S31508002090452F0008452F0008452F0008452F000842
S315080020A0452F0008452F0008452F0008452F000832
S315080020B0452F0008452F000800000000452F00089E
S315080020C0452F00080000000000000000452F00080A
S315080020D000000000452F0008452F0008452F00087E
S315080020E0452F0008452F00080000000000000000EA
S315080020F000000000000000000000000000000000D2
S3150800210000000000000000000000000000000000C1
S315080021100000000000000000452F0008452F0008B9
S3150800212000000000000000000000000000000000A1
S315080021300000000000000000000000000000000091
S31508002140452F0008452F0008000000000000000089
S315080021500000000000000000000000000000000071
S315080021600000000000000000000000000000000061
S315080021700000000000000000000000000000000051
S3110800218000000000452F0008EE11AA55CB
S3150800218C10B5054C237833B9044B13B10448AFF397
S3150800219C00800123237010BD3400002000000000CD
S315080021ACFC2F000808B5034B1BB103490348AFF3D2
S315080021BC008008BD0000000038000020FC2F000835
S315080021CCF0B5002401E00134E4B2112C20D8114DED
S315080021DC15F814E005EB44056F780EEB070606FBBD
S315080021EC00064FF4FA4595FBF6F506FB05F5B5F52D
S315080021FCFA4FE8D195FBF6F6B6B20E80013EB6B2AA
S3150800220CB6F5806FDFD282F800E01F700120F0BDB2
S3150800221C0020F0BD1430000870B588B001214FF4C9
S3150800222C003000F055FD01214FF4003000F042FD5E
S3150800223C072202214FF0904000F06CFB07220F2179
S3150800224C4FF0904000F066FB00248DF81E400125E7
S3150800225C8DF81F5002268DF81C6004230693032361
S3150800226C8DF81D3006A94FF0904000F007FB8DF84D
S3150800227C1C604FF40043069306A94FF0904000F0FB
S3150800228CFDFA4FF461430093019402940394059468
S3150800229C0C230493054C6946204600F035FD294667
S315080022AC204600F095FD08B070BD00BF0044004004
S315080022BC70B58AB001214FF4003000F0FBFC0922FE
S315080022CC0B214FF0904000F025FB09220C214FF012
S315080022DC904000F01FFB4FF4C053089302238DF86F
S315080022EC243003238DF8253000248DF8264001254B
S315080022FC8DF8275008A94FF0904000F0BFFA2946F0
S3150800230C4FF0007000F0E4FC244E304600F02AF939
S3150800231C05A800F043FA6B460DEB05020DF1020118
S3150800232C4FF4FA70FFF74CFF8DF81A408DF81B40E6
S3150800233C8DF81C408DF81D408DF81E408DF81F40F9
S3150800234C8DF816408DF817409DF80130013B8DF835
S3150800235C18309DF80030013B8DF81930BDF8023065
S3150800236CADF8143005A9304600F008F98DF80E4082
S3150800237C8DF80F408DF81050ADF80440ADF80640B6
S3150800238CADF80840ADF80A40ADF80C408DF8115080
S3150800239C01A800F085F90AB070BD00BF00640040C2
S315080023AC10B504462021064800F021FD012801D06D
S315080023BC002010BD024800F016FD2070012010BD4B
S315080023CC0044004008B5FFF727FFFFF771FF08BD6B
S315080023DCBFF34F8F0449CA6802F4E062034B1343F8
S315080023ECCB60BFF34F8FFEE700ED00E00400FA0563
S315080023FC08B5214B1B78A3B92048FFF7D1FF012854
S3150800240C00D008BD1D4B1B78002BFAD000F0BEFD82
S3150800241C1B4B18600122184B1A700022194B1A70A4
S3150800242C08BD184B1B78013314481844FFF7B8FF3E
S3150800243C01280AD000F0AAFD114B1B686433984298
S3150800244CDFD900220C4B1A70DBE70E4A13780133DE
S3150800245CDBB21370094A12789342D2D10022064B8A
S3150800246C1A70064B5B78FF2BCBD1044B9B78002B51
S3150800247CC7D1FFF7ADFF00BF910000205000002028
S3150800248C940000209200002000B587B000210D486A
S3150800249C00F0E7F910B907B05DF804FB01AA0021B2
S315080024AC084800F08BF940F26763019A9A42F2D118
S315080024BC9DF80F30FF2BEED19DF81030002BEAD18A
S315080024CCFFF786FF0064004008B5FFF791FFFFF79A
S315080024DCDBFF08BD30B583B001214FF4802000F036
S315080024ECE9FB0825009501238DF8043000238DF8A7
S315080024FC063003228DF805208DF80730054C694601
S3150800250C204600F0BBF92946204600F001FA03B034
S3150800251C30BD00BF0004004810B500F037FD0E4B67
S3150800252C1B68C31AB3F5FA7F0CD304460B4B1B78FE
S3150800253C4BB90122094B1A700821094800F0E6F933
S3150800254C054B1C6010BD0022044B1A700821044868
S3150800255C00F0DEF9F4E700BF9C000020980000208C
S3150800256C0004004808B501214FF0007000F0BEFBCE
S3150800257C00214FF0007000F0B9FB08BD82B00023B3
S3150800258C0193036823F002030360036843F0010315
S3150800259C036002E0019B01330193436813F0010FBA
S315080025AC04D1019A6FF07F439A42F3D1436813F032
S315080025BC010F71D08B79012B3CD0036823F0800373
S315080025CC0360CB79012B3AD0036823F040030360F0
S315080025DC0B7A012B38D0036823F0200303604B7A5F
S315080025EC012B36D0036823F0100303608B7A012B7A
S315080025FC34D0036823F008030360CB7A012B32D05E
S3150800260C036823F0040303608A78CB781B0643EA35
S3150800261C82730A7943EA02434A7943EA02530A88DF
S3150800262C013A1343C361036823F0010303600023D3
S3150800263C019320E0036843F080030360C1E7036855
S3150800264C43F040030360C3E7036843F020030360C9
S3150800265CC5E7036843F010030360C7E7036843F054
S3150800266C08030360C9E7036843F004030360CBE778
S3150800267C019B01330193436813F0010F04D0019AAF
S3150800268C6FF07F439A42F3D1436813F0010F01D1DF
S3150800269C012002E0002000E0002002B07047000094
S315080026AC70B4837A012202FA03F33B4AD2F8001279
S315080026BC41F00101C2F80012D2F81C42D9430C4071
S315080026CCC2F81C42027BB2B9334AD2F80C420C400F
S315080026DCC2F80C42847AC688458845EA06454834C9
S315080026EC42F83450857A8688048844EA0644483584
S315080026FC02EBC5025460027B012A1FD0C27A002A5B
S3150800270C34D1254CD4F804220A40C4F80422028990
S3150800271C2AB9214AD2F814422140C2F81412028965
S3150800272C012A2AD0427B012A2ED01B4AD2F8003223
S3150800273C23F00103C2F8003270BC7047164AD2F86F
S3150800274C0C421C43C2F80C42847A0688458845EA32
S3150800275C0645483442F83450857A8688C48844EA53
S3150800276C0644483502EBC5025460C7E70A4CD4F850
S3150800277C04221A43C4F80422C9E70749D1F81422DB
S3150800278C1A43C1F81422CDE7034AD2F81C120B439C
S3150800279CC2F81C32C9E700BF0064004000238371ED
S315080027ACC371037243728372C3728370C37003233B
S315080027BC03710223437101230380704710B401F19E
S315080027CC1B031B01C35803F004031372002B3CD1E3
S315080027DC01F11B031B01C3585B0D136001F11B03AD
S315080027EC1B01C418C35803F002035372636803F041
S315080027FC0F03937263681B0AD37400EB0113D3F8A7
S3150800280CB841D472D3F8B841240A1473D3F8B84132
S3150800281C240C5473D3F8B841240E9473D3F8BC41E2
S3150800282CD473D3F8BC41240A1474D3F8BC41240CD1
S3150800283C5474D3F8BC311B0E937469B1036943F015
S3150800284C200303615DF8044B704701F11B031B0160
S3150800285CC358DB085360C1E7C36843F02003C36061
S3150800286CF0E719B1012905D000207047C06800F0BF
S3150800287C03007047006900F00300704700230F2B14
S3150800288C43D8F0B434E085685F000326BE4025EAD9
S3150800289C0605856082684C79BC402243826085882F
S315080028ACADB29FB20126BE4025EA06058580828810
S315080028BC92B28C79BC40A4B22243828002685D0035
S315080028CC032404FA05F622EA0602026002680E7967
S315080028DCAE4032430260C2689EB27600B44022EA29
S315080028EC0402CC79AC402243C26001330F2B0AD8C0
S315080028FC01229A400C68A243F7D10A79013AD2B25E
S3150800290C012ADBD8BFE7F0BC704770478161704776
S3150800291C0185704730B401F007039B009A40C9083B
S3150800292C083150F821400F2505FA03F324EA03036E
S3150800293C40F8213050F821301A4340F8212030BC99
S3150800294C70470000F0B5A04B5A6802F00C02042A36
S3150800295C3AD0082A3CD01AB19C4B0360002201E0FD
S3150800296C9A4B0360984D6B68C3F30313DFF864E264
S3150800297C1EF80370FFB2016821FA07F343606C680E
S3150800298CC4F302241EF80440E4B223FA04F4846067
S3150800299C6E68C6F3C2261EF80660F6B2F340C3602C
S315080029ACED6A2D0905F00F0CDFF82CE23EF81CE059
S315080029BC1FFA8EFE15F0100F23D0BEF1000F20D093
S315080029CCB2FBFEF505611DE0804B03600022C9E7EA
S315080029DC7D4B5A685B68C2F38342023213F4803F1C
S315080029EC04D17B4B03FB02F20260BBE7764BDB6A36
S315080029FC03F00F0301337549B1FBF3F303FB02F242
S31508002A0CF2E70161704DED6A6D0A05F00F0CDFF8FF
S31508002A1CC8E13EF81CE01FFA8EFE15F0100F06D022
S31508002A2CBEF1000F03D0B2FBFEF5456100E0416133
S31508002A3C654D2D6B15F0100F40F08180634D856147
S31508002A4C614D2D6B15F0200F7BD1604DC5615E4D28
S31508002A5C2D6B15F0400F76D15C4D05625A4D2D6BDA
S31508002A6C15F4807F01D08A426FD04362564D2D6B88
S31508002A7C15F4805F01D08A426CD08362524D2D6B5F
S31508002A8C15F4007F01D08A4269D0C3624E4D2D6B76
S31508002A9C15F4806F01D08A4266D0C3644A4D2D6BFB
S31508002AAC15F4006F01D08A4263D00365464D2D6B31
S31508002ABC15F4005F01D08A4260D00365424D2D6B38
S31508002ACC15F4004F01D08A425DD083653E4B1B6BD3
S31508002ADC13F0030F5CD184633B4B1B6B13F4403F21
S31508002AEC7CD1C463384B1B6B13F4402F40F0958094
S31508002AFC0464354B1B6B13F4401F40F0AD804464E3
S31508002B0C314B1B6B13F4400F00F0C5802E4B1B6B1F
S31508002B1C03F44003B3F5800F00F0BF802A4B1B6B00
S31508002B2C03F44003B3F5000F00F0B980264B1B6B7A
S31508002B3C03F44003B3F5400F00F0B580F0BD816196
S31508002B4C7EE7C16183E7016288E7B7428DD15500FC
S31508002B5C45628BE7B74290D1550085628EE7B7423E
S31508002B6C93D15500C56291E7B74296D15500C56415
S31508002B7C94E7B74299D15500056597E7B7429CD1BA
S31508002B8C550045659AE7B7429FD1520082659DE785
S31508002B9C0D4B1B6B03F00303012B0ED00A4B1B6B5F
S31508002BAC03F00303022B0AD0074B1B6B03F003033A
S31508002BBC032B91D1054B83638EE781638CE74FF426
S31508002BCC0043836388E700BF0010024000127A00B6
S31508002BDC00093D002000002000000020334B1B6B31
S31508002BEC03F44033B3F5803F11D0304B1B6B03F421
S31508002BFC4033B3F5003F0CD02C4B1B6B03F440331E
S31508002C0CB3F5403F7FF46EAF294BC3636AE7C163E4
S31508002C1C68E74FF40043C36364E7244B1B6B03F468
S31508002C2C4023B3F5802F11D0204B1B6B03F44023A4
S31508002C3CB3F5002F0CD01D4B1B6B03F44023B3F5D7
S31508002C4C402F7FF456AF1A4B036452E7016450E7E2
S31508002C5C4FF4004303644CE7144B1B6B03F440130B
S31508002C6CB3F5801F11D0114B1B6B03F44013B3F54E
S31508002C7C001F0CD00D4B1B6B03F44013B3F5401F10
S31508002C8C7FF43EAF0A4B43643AE7416438E74FF4A6
S31508002C9C0043436434E78464F0BD8164F0BD4FF4AB
S31508002CAC00438364F0BD024B836447E7001002407F
S31508002CBC00127A0029B9054A536923EA00005061C3
S31508002CCC7047024A53691843506170470010024016
S31508002CDC29B9054AD36923EA0000D0617047024A2C
S31508002CECD3691843D06170470010024029B9054AC8
S31508002CFC136923EA000010617047024A13691843E6
S31508002D0C106170470010024030B599B004460D4664
S31508002D1C036823F001030360436823F440538A686D
S31508002D2C13434360036823F4B05323F00C034A6837
S31508002D3CC9680A4329690A4313430360836823F461
S31508002D4C40736A691343836001A8FFF7FBFD1C4BAC
S31508002D5C9C4227D01B4B9C4226D01B4B9C4225D011
S31508002D6C1A4B9C4224D01399236813F4004F21D094
S31508002D7C49002A68B1FBF2F302FB13122968B2EB7D
S31508002D8C510F00D30133226812F4004F06D0C3F357
S31508002D9C420223F00F031B041B0C13439BB2A381A3
S31508002DAC19B030BD0F99DFE71099DDE71199DBE70C
S31508002DBC1299D9E72A68B1FBF2F302FB1312DDE785
S31508002DCC003801400044004000480040004C0040D8
S31508002DDC21B9036823F0010303607047036843F0C5
S31508002DEC010303607047808CC0F308007047C36901
S31508002DFC0B4201D100207047012070471222164B56
S31508002E0C1A60A3F580535A685A605A685A605A6809
S31508002E1C42F480625A605A6822F47C125A605A68E4
S31508002E2C42F460125A601A6842F080721A600B4BB0
S31508002E3C1B6813F0007FFAD0084B5A6822F003027D
S31508002E4C5A605A6842F002025A60044B5B6803F0F7
S31508002E5C0C03082BF9D170470020024000100240E1
S31508002E6C08B5154AD2F8883043F47003C2F888308E
S31508002E7C124B1A6842F001021A605968104A0A4045
S31508002E8C5A601A6822F0847222F480321A601A6820
S31508002E9C22F480221A605A6822F4FE025A60DA6A10
S31508002EAC22F00F02DA62196B064A0A401A630022EC
S31508002EBC9A60FFF7A3FF08BD00ED00E00010024082
S31508002ECC0CC07FF8CCFC00FF08B5FFF703FB00F03D
S31508002EDC3BF808BD08B5FFF7F7FFFFF773FAFFF7DE
S31508002EEC1BFBFFF7F1FAFAE7DFF834D0002103E011
S31508002EFC0C4B5B58435004310B480C4B42189A4206
S31508002F0CF6D30B4A02E0002342F8043B094B9A42DB
S31508002F1CF9D3FFF7A5FF00F047F8FFF7DBFFFEE74D
S31508002F2C003000204030000800000020340000204B
S31508002F3C34000020A4000020FEE70000014B1860B6
S31508002F4C704700BFA000002008B50C4B1B680C4A44
S31508002F5CA2FB03239B09013BB3F1807F09D2094AE3
S31508002F6C5360F021084B83F8231000239360072342
S31508002F7C13600020FFF7E2FF08BD00BF30000020F9
S31508002F8CD34D621010E000E000ED00E0014B18682C
S31508002F9C704700BFA0000020024A13680133136073
S31508002FAC704700BFA000002070B50D4E0D4CA41B39
S31508002FBCA4100025A54209D10B4E0C4C00F018F8AC
S31508002FCCA41BA4100025A54205D170BD56F82530C2
S31508002FDC98470135EEE756F8253098470135F2E75C
S31508002FEC3830000838300008383000083C30000803
S31508002FFCF8B500BFF8BC08BC9E467047F8B500BFCC
S30D0800300CF8BC08BC9E4670479B
S3150800301405020602060307030803090309040A044A
S315080030240B040C040C050D050E050F050F061006FA
S30908003034100710085B
S30908003038B1210008AC
S3090800303C8D210008CC
S31508003040010002000400060008000A000C00100037
S315080030502000400080000001000000000000000081
S315080030600000000001020304010203040607080920
S309080030700090D003EB
S70508002EF5CF
